:020000020000FC
:1000000000C002E00EBF0FE50DBF0FEF04BB00E024
:1000100005BB0E94280007E40E94820005E60E94BA
:10002000820008E60E94820004E70E94820000EC41
:100030000E946D000CE40E94820001E60E94820092
:100040000CE60E94820001E60E9482000C942600C9
:100050000E94CF000E94CF0000E30E9461000E9436
:10006000CF0000E30E9461000E94CF0000E30E94E5
:1000700061000E94CF0000E20E9461000E94CF0058
:1000800008E20E946D000E94CF000CE00E946D000B
:100090000E94CF0001E00E946D000E94CF0006E0A8
:1000A0000E946D000E94CF00089501E00E946D0043
:1000B0000E94CF00089502E00E946D000E94CF00D0
:1000C00008950E949700A898A9980000A89A000097
:1000D0000000A8980E94090108950E949700A8981E
:1000E000A9980000A89A00000000A8980E940901A1
:1000F0000E94A4000000A89A00000000A8980E9496
:10010000090108950E949700A898A99A0000A89A4A
:1001100000000000A8980E9409010E94A4000000AD
:10012000A89A00000000A8980E9409010895AE98BE
:10013000AD98AC98AB9807FDAE9A06FDAD9A05FD5B
:10014000AC9A04FDAB9A0895AE98AD98AC98AB9874
:1001500003FDAE9A02FDAD9A01FDAC9A00FDAB9A8B
:1001600008950E94C3000E94C3000E94C3000E9421
:10017000C3000E94C3000E94C3000E94C3000E94EB
:10018000C3000E94C3000E94D9000E94CF000E94B9
:10019000CF000E94CF000E94CF000E94CF000E949B
:1001A000EB000E94EB000E94EB000E94EB000E941B
:1001B000EB000E94EB000E94EB000E94EB000E940B
:1001C000EB000E94EB000E94EB000E94EB000E94FB
:1001D000EB000E94EB000E94FD000E94FD000E94C7
:1001E000FD000E94FD000E94FD000E94FD000E9493
:1001F000FD000E94FD000E94FD000E940F010E9470
:100200000F010E940F010E940F010E940F010E9426
:100210000F010E940F010E940F010E940F010E9416
:1002200021010E9421010E9421010E9421010E94BE
:1002300021010E9421010E9421010E9421010E94AE
:10024000210100000000000000000000000000008C
:0E025000000000000000000000000000089503
:00000001FF
